:10000000FFC1FFC1FFC1FFC1FFC1FFC1FFC1FFC1F0
:10001000FFC1FFC1FFC1FFC1FFC1FFC1FFC1FFC1E0
:10002000FFC1FFC1FFC1FFFFFFFFFFFFFFFFFFFF9A
:10003000FFFFFFFFFFFFFFFFFFFFFFFFFFFFFFFFD0
:10004000FFFFFFFFFFFFFFFFFFFFFFFFFFFFFFFFC0
:10005000FFFFFFFFFFFFFFFFFFFFFFFFFFFFFFFFB0
:10006000FFFFFFFFFFFFFFFFFFFFFFFFFFFFFFFFA0
:10042000FFC1FFC1FFC1FFFFFFFFFFFFFFFFFFFF96
:10043000FFFFFFFFFFFFFFFFFFFFFFFFFFFFFFFFCC
:10044000FFFFFFFFFFFFFFFFFFFFFFFFFFFFFFFFBC
:10045000FFFFFFFFFFFFFFFFFFFFFFFFFFFFFFFFAC
:10046000FFFFFFFFFFFFFFFFFFFFFFFFFFFFFFFF9C
:10082000FFC1FFC1FFC1FFFFFFFFFFFFFFFFFFFF92
:10083000FFFFFFFFFFFFFFFFFFFFFFFFFFFFFFFFC8
:10084000FFFFFFFFFFFFFFFFFFFFFFFFFFFFFFFFB8
:10085000FFFFFFFFFFFFFFFFFFFFFFFFFFFFFFFFA8
:10086000FFFFFFFFFFFFFFFFFFFFFFFFFFFFFFFF98
:100C00001EC152C137C136C135C134C133C132C131
:100C100031C130C12FC12EC12DC12CC12BC12AC160
:100C200029C128C127C105010906A101750195083F
:100C3000050719E029E715002501810295017508CE
:100C40008103950575010508190129059102950192
:100C500075039103950675081500256505071900AC
:100C600029658100C00902220001010080320904C7
:100C700000000103010100092101010001223F00E0
:100C80000705810308000A12011001000000084254
:100C90004231E10001010200011A03740069006E93
:100CA00000790055005300420062006F006100723D
:100CB000006400520368007400740070003A002F52
:100CC000002F006D006100740072006900780073ED
:100CD0000074006F0072006D002E0063006F006DE5
:100CE000002F006100760072002F00740069006E12
:100CF00000790075007300620062006F006100728D
:100D00000064002F000403090474696E795553428E
:100D1000626F617264205265762E330A6874747053
:100D20003A2F2F6D617472697873746F726D2E63D0
:100D30006F6D2F6176722F74696E79757362626F51
:100D40006172642F0A0A0A42656920416E6D6572FC
:100D50006B756E67656E2C2046726167656E206FDD
:100D60006465722050726F626C656D656E20776588
:100D70006E64656E205369652073696368206269DB
:100D800074746520616E205374657068616E2042D2
:100D9000616572776F6C660A7374657068616E4026
:100DA0006D617472697873746F726D2E636F6D2CE0
:100DB000206D617472697873746F726D40676D78BD
:100DC0002E64652C207374657068616E2E62616597
:100DD00072776F6C664074752D696C6D656E6175A8
:100DE0002E64650A0A5047502D4B65794944093AEB
:100DF00020307846423942313244420A46696E67B1
:100E000065727072696E74093A203232353220424E
:100E10003431452031324446203431414420343786
:100E20003646203746333620303834412030393189
:100E300031204642394220313244420A0000112416
:100E40001FBECFE5D4E0DEBFCDBF10E0A0E6B0E02E
:100E5000E4EBF7E102C005900D92A636B107D9F791
:100E600020E0A6E6B0E001C01D92AA3AB207E1F781
:100E700033D29EC4C5CEA82FB92F80E090E041E0C8
:100E800050EA609530E009C02D91822797958795AB
:100E900010F084279527305EC8F36F5FA8F308959C
:100EA000EADF8D939D930895CF93CFB7CF93DF93D0
:100EB000C395879BE9F7879B0BC0879B09C0879BDE
:100EC00007C0879B05C0879B03C0879B01C08BC061
:100ED0006F93C0918D00DD27CC56DF4F2F9365E5D2
:100EE000879B03C02F916F91E6CF0F931F934F9372
:100EF00020E040E15F9300B3047807FB27F93F93BC
:100F000050E03BE039C0147840642F77012F5F5FD9
:100F10001EC0406810B314782F7752501FC0406431
:100F200000B32F770478D1F15F5F00C023C0406227
:100F300010B32F77147891F15F5F00C025C004785B
:100F40001027515012F45D5F0000115027952C3F7F
:100F500010B3C8F614780127015027952C3FC8F626
:100F60004227499300B3047810274F7311502795F7
:100F70002C3FA8F64695469510B3147879F00127D2
:100F8000015027952C3F98F66B5A60F3315000B30F
:100F9000B0F600C010E41ABF002719C03B503195CD
:100FA000C31BD04010E41ABF0881033C09F10B3485
:100FB000F9F020918B001981110F1213EDCF4A81A6
:100FC000441F093651F10D3211F0013E29F700930B
:100FD00092003F915F914F911F910F912F916F91CF
:100FE000CAB7C6FD65CFDF91CF91CFBFCF9118951E
:100FF00020919200222369F310919000112391F522
:10100000343092F13093900020938C0010918D0039
:101010003BE0311B30938D0027C0009190000130E0
:101020000CF50AE54F7049F43091610034FD1DC0A4
:1010300000936100C4E7D0E01CC030917F0034FD14
:1010400014C000937F00C0E8D0E013C0052710E073
:1010500000C0000002BB1AC0052710E0221F1DC0FF
:1010600010E021C04AE502C032ED432FC4E1D0E0D8
:1010700032E011B31468979A02B311BB54E820E828
:1010800065E320FF052702BB279517951C3FF0F667
:101090006695B8F7B1F720FF052702BB279517958E
:1010A0001C3FD0F62795179517FF052700001C3F1A
:1010B00002BBB0F629913A9519F70B771091910080
:1010C000110FC651D04002BB11F010938B0010E4F9
:1010D0001ABF006811B31B77402F4B7754E05A9525
:1010E000F1F702BB11BB42BB74CF20917F0024FFFC
:1010F00007C02091800038E823272093800003C098
:101100002AE520937F00FC01A1E8B0E081918D9356
:1011100080E0A938B807D1F768E081E890E0C0DE48
:101120008CE080937F000895FC0188E0DF011D9230
:101130008A95E9F708958091620090916300019685
:10114000C9F088B392E0892788BB8091600080FF56
:1011500002C0939A01C093988091600081FF02C001
:10116000959A01C095988091600082FF02C0C09A54
:101170000895C09808951F93CF93DF93CDB7DEB73E
:1011800060970FB6F894DEBF0FBECDBF182FCE010B
:101190000996CADF103211F48CE254C01A3011F4EF
:1011A00088E250C0193011F48BE24CC01A3709F4B0
:1011B00004C01A3521F482E089878CE143C01937D5
:1011C00009F404C0193521F482E089878DE13AC021
:1011D000812F81568A3110F41D550DC0812F815405
:1011E0008A3120F482E089871D5305C0812F815305
:1011F000893018F413511B8726C0103311F487E28D
:1012000021C0103419F4198784E11CC01A3319F471
:1012100082E0898716C01C3211F486E313C01F32A6
:1012200011F484E50FC01A3211F485E50BC01B32AE
:1012300011F487E507C01D3211F486E503C01E32A4
:1012400011F487E38B8788E0FE013996DE01119661
:1012500001900D928A95E1F729813A814B815C8159
:101260006D817E818F81988560960FB6F894DEBF80
:101270000FBECDBFDF91CF911F910895CF93DF9324
:10128000CDB7DEB760970FB6F894DEBF0FBECDBF07
:101290008FEF71DF29873A874B875C876D877E8761
:1012A0008F87988B88E0FE013996DE0111960190B8
:1012B0000D928A95E1F729813A814B815C816D819C
:1012C0007E818F81988560960FB6F894DEBF0FBE41
:1012D000CDBFDF91CF910895CF93DF93CDB7DEB728
:1012E00060970FB6F894DEBF0FBECDBF2FE088E148
:1012F00090E00FB6F894A89581BD0FBE21BD85B7CB
:10130000836085BF8BB780648BBF8BE48093800044
:101310008AE580937F008F9AA8958B9A8D9AB89AC8
:10132000B99A96988E98969A2FEF83EC99E021506F
:1013300080409040E1F700C00000A8958F98789415
:10134000A89580919000835087FDEFC090918D000B
:101350000CE010E0091B11090C561F4F90918C00F6
:101360009D3209F0D1C0883009F0DDC083EC809354
:1013700074008AE58093610010926B00F80180810F
:10138000807661F1803241F581818230C9F018F4B4
:10139000813011F505C0893061F08A30E9F418C058
:1013A0008CE690E090938F0080938E00BDDE28E065
:1013B000A0C0F80186819781019771F42FEF91C049
:1013C0008AE690E090938F0080938E0021E091C098
:1013D000F801838180936A0020E08BC0F80192813C
:1013E00010927D008181811106C010927E008DE7F0
:1013F00090E022E070C0853019F49093910068C0AD
:10140000863009F04FC0F8018381813041F487E8CC
:101410009CE090938F0080938E0022E13FC0823049
:1014200041F485E69CE090938F0080938E0022E249
:1014300035C08330F1F4911108C085E09DE09093B0
:101440008F0080938E0024E029C0913041F483EB1B
:101450009CE090938F0080938E0022E51FC0923015
:10146000E1F489E99CE090938F0080938E002AE15B
:1014700015C0813241F487E79CE090938F00809300
:101480008E0029E00BC0823241F486E29CE090930A
:101490008F0080938E002FE301C020E080E48093D2
:1014A0006B001DC0883069F0893019F49093930067
:1014B0000FC08A3049F08B3059F48BE48093800060
:1014C00007C083E990E002C08DE790E021E003C00F
:1014D0008DE790E020E090938F0080938E002F3F67
:1014E00041F4F801808187FD268180E880936B00BC
:1014F00008C0F8018781811104C08681821708F431
:10150000282F209364000FC080916B0087FF0BC0D1
:10151000F801808190916000891719F08093600034
:101520000ADE10926400109290008091610084FFA6
:1015300043C0809164008F3F09F43EC0182F89306A
:1015400008F018E0811B809364008091740098E893
:10155000892780937400112319F1E0918E00F09196
:101560008F0080916B0086FF0BC0A5E7B0E08491EF
:101570008D93319685E790E0810F8A13F8CF0CC0E8
:10158000CF01A5E7B0E0FC012191CF012D9325E724
:1015900030E0210F2A13F7CFF0938F00E0938E00F5
:1015A000612F85E790E07CDC1C5F1C3019F08FEF29
:1015B000809364001093610084E190B3947831F4D7
:1015C0008150D9F71092910010928B0080917F008A
:1015D00084FFACC080916200909163000196C1F5D8
:1015E000C0906600D0906700E0906800F0906900BD
:1015F00020EAC21626E8D20621E0E206F104D8F479
:10160000C701B60122E03DE040E050E0AFD0672BDB
:10161000682B692B81F488B392E0892788BB82B359
:1016200098E0892782BB82B390E2892782BB88B386
:1016300091E0892788BB80EAC81686E8D80681E051
:10164000E806F10428F0109263001092620073DD46
:10165000E0906200F09063008701169507950333D0
:1016600091E0190708F05BC0E0FE16C007DE29878D
:101670003A874B875C876D877E878F87988B88E05A
:10168000FE013996DE01119601900D928A95E1F7DF
:10169000EFEFEE1AFE0A3BC080916A00F4E08F9FE4
:1016A000C00111248233910510F482E390E04AE0F6
:1016B000489F9001499F300D1124442737FD4095E4
:1016C000542F60916600709167008091680090913E
:1016D00069004CD0672B682B692B41F5F801E75F57
:1016E000F24F849148DD29873A874B875C876D8765
:1016F0007E878F87988B88E0FE013996DE011196F0
:1017000001900D928A95E1F72FEFE21AF20AF0921A
:101710006300E0926200CE010196E7DC07C0869983
:1017200005C0109263001092620005DD8091660092
:1017300090916700A0916800B09169000196A11D89
:10174000B11DB7FF04C0B695A7959795879580936F
:10175000660090936700A0936800B09369008FE8DB
:1017600091E00197F1F700C00000EACDA1E21A2E46
:10177000AA1BBB1BFD010DC0AA1FBB1FEE1FFF1F35
:10178000A217B307E407F50720F0A21BB30BE40B85
:10179000F50B661F771F881F991F1A9469F76095CC
:1017A0007095809590959B01AC01BD01CF01089586
:1017B000F894FFCFFF5AFFFFFF00FFFFFFFFFFFF7F
:1017C000FFFFFFFFFFFFFFFFFFFFFFFFFFFFFFFF29
:1017D000FFFFFFFFFFFFFFFFFFFFFFFFFFFFFFFF19
:1017E000FFFFFFFFFFFFFFFFFFFFFFFFFFFFFFFF09
:1017F000FFFFFFFFFFFFFFFFFFFFFFFFFFFF0000F7
:101800005DC0ADC082C081C080C07FC07EC07DC0D1
:101810007CC07BC07AC079C078C077C076C075C004
:1018200074C073C072C07E3FF9F76A39F9F7563554
:10183000F9F74038F9F7EC2DFD2DB7B6B0FCFDCF28
:1018400027BFE895B7B6B0FCFDCF21E1B7B6B6FC2F
:10185000F4CF089576302E3937205374657068615F
:101860006E2042616572776F6C6609021200010199
:101870000080320904000000000000001201100185
:10188000FF000008C016DC050201010200010E0382
:101890005500530042006100730070001C03770084
:1018A000770077002E00660069007300630068000F
:1018B0006C002E00640065000403090411241FBE9F
:1018C000CFE5D4E0DEBFCDBF24B7D4E0CEE539917B
:1018D0003C30399109F03FEF30939B0020939A0000
:1018E00010E0A0E6B0E0EAEFFFE102C005900D9243
:1018F000A636B107D9F720E0A6E6B0E001C01D92F8
:10190000AA39B207E1F789D176C37ACFA82FB92FC8
:101910008FEF9FEF1BC02D918227282F229528271C
:10192000722F269526952727239526952170782FA7
:10193000892F82272195207C922F22277695279523
:10194000972782277695279597278227615018F742
:10195000809590950895DADF8D939D930895CF93A8
:10196000CFB7CF93DF93C395879BE9F7879B0BC0D6
:10197000879B09C0879B07C0879B05C0879B03C0C7
:10198000879B01C089C06F93C0917D00DD27CC5734
:10199000DF4F2F9365E5879B03C02F916F91E6CFB3
:1019A0000F931F934F9320E040E15F9300B30478BF
:1019B00007FB27F93F9350E03BE039C014784064BF
:1019C0002F77012F5F5F1EC0406810B314782F7708
:1019D00052501FC0406400B32F770478D1F15F5F8D
:1019E00000C023C0406210B32F77147891F15F5F7D
:1019F00000C025C004781027515012F45D5F00002C
:101A0000115027952C3F10B3C8F6147801270150C8
:101A100027952C3FC8F64227499300B30478102736
:101A20004F73115027952C3FA8F64695469510B355
:101A3000147879F00127015027952C3F98F66B5ABE
:101A400060F3315000B3B0F600C010E41ABF0027B5
:101A500017C03B503195C31BD04010E41ABF08811A
:101A6000033CF9F00B34E9F020917B001981110F50
:101A70001213EDCF093651F10D3211F0013E39F755
:101A8000009382003F915F914F911F910F912F9191
:101A90006F91CAB7C6FD67CFDF91CF91CFBFCF910E
:101AA000189520918200222369F310918000112360
:101AB00039F534303AF13093800020937C00109156
:101AC0007D003BE0311B30937D001CC00091800005
:101AD0000130B4F40AE53091610034FD14C0009384
:101AE0006100C0E7D0E013C0052710E000C000008F
:101AF00002BB1AC0052710E0221F1DC010E021C044
:101B00004AE502C032ED432FC4E1D0E032E011B328
:101B10001468979A02B311BB54E820E865E320FFEC
:101B2000052702BB279517951C3FF0F66695B8F779
:101B3000B1F720FF052702BB279517951C3FD0F66C
:101B40002795179517FF052700001C3F02BBB0F62D
:101B500029913A9519F70B7710918100110FC65111
:101B6000D04002BB11F010937B0010E41ABF006854
:101B700011B31B77402F4B7754E05A95F1F702BB16
:101B800011BB42BB7FCFF8948F9A96981BBE15BEAF
:101B9000F1E0FBBF1BBE34C2FC013381932F4481B3
:101BA000842F2281203339F44370E42FF0E0EE5982
:101BB000FF4F80810895283529F431110EC0E1E0EE
:101BC000F0E006C0203571F4311125C0E0E0F0E00E
:101BD00089E080935700849108953830E1F4E3E080
:101BE000F0E0F6CF203221F4FC01EE0FFF1F06C01B
:101BF000283231F4FC01EE0FFF1F319684910895D5
:101C0000203A09F4E3C1203C19F46581E7D103C00F
:101C10002F3F09F411EF80E0089511BA80E482BBF0
:101C200081E08BBF82E08BBF84E031978040E9F791
:101C300080919A00877F21F480919B00882311F086
:101C40008699A1DF1EEF14BE85B7826085BF8BB772
:101C500080648BBF8F9A80E131978040E9F78F983D
:101C6000789400918000035007FD2BC180917D0086
:101C7000CCE0D0E0C81BD109CC57DF4F80917C006D
:101C80008D3209F0B5C0083009F019C183EC80939A
:101C900070008AE58093610010926F004881842F64
:101CA00080763981882399F186E690E090937F00D1
:101CB00080937E00333031F4CE016EDF8093690073
:101CC00024E08CC03530F9F03A30E9F08CEF830F26
:101CD000863098F48A819B8190936E0080936D008A
:101CE000393099F08E8180936C008D818270809361
:101CF0006B0030936A002FEF6BC0323011F41E7FFF
:101D000004C0116002C021E069C020E067C08A8180
:101D100010927900311106C010927A0089E790E0A4
:101D200022E050C0353019F4809381003DC0363038
:101D3000A9F59B81913019F48CE798E104C09230A9
:101D400041F48AE698E190937F0080937E0022E13F
:101D500021C09330F1F4811108C088EB98E1909391
:101D60007F0080937E0024E015C0813041F48CE92F
:101D700098E190937F0080937E002CE10BC082302D
:101D800041F48EE898E190937F0080937E002EE0EE
:101D900001C020E080E480936F0018C0383079F0F3
:101DA000393031F48093830089E790E020E00AC065
:101DB00021E03A3009F020E089E790E003C083E8B1
:101DC00090E021E090937F0080937E002F3F31F4DC
:101DD00047FD2E8180E880936F0007C08F818111BD
:101DE00004C08E81821708F4282F2093600067C0FA
:101DF00080916F0087FF63C080916C00801708F4AA
:101E0000082F801B80936C00DD24D3948111D12C8A
:101E100080916A008730C0F0CC2EEC2EFD2E8E2DE6
:101E20008C19801708F048C0D7016D917D01809111
:101E30006D0090916E009C012F5F3F4F30936E00BC
:101E400020936D00CBD0EBCF80916B00E0916D00C3
:101E5000F0916E00DE0100FD0395025048F1F8316B
:101E600038F522D0F8940D901D9021E017D02E2F38
:101E70002E5F2F7331F0DD2079F0882369F0003078
:101E800059F423E00BD010D025E008D00DD007B6D0
:101E900006FE02C021E102D03296DFCFF89427BFC0
:101EA000E89511247894089507B600FCFDCF0895B5
:101EB000F0936E00E0936D00D110109260001092CC
:101EC00080008091610084FF6BC0809160008F3F33
:101ED00009F466C0082F893008F008E0801B809361
:101EE00060008091700098E889278093700000233B
:101EF00009F44AC080916F0087FF28C080916C0070
:101F0000801708F4082F801B80936C00D0906A0023
:101F1000C1E7D0E081E790E02C2F281B2017A0F527
:101F2000E0906D00F0906E00B6E0BD1518F4C701AA
:101F30004DD002C0F701849188832196FFEFEF1AFC
:101F4000FF0AF0926E00E0926D00E4CFE0917E0017
:101F5000F0917F0086FF0BC081E790E0DC012491C7
:101F60002D933196202F280F2A13F9CF09C081E72E
:101F700090E0DC0121912D93202F280F2A13FACF16
:101F8000F0937F00E0937E00602F81E790E0E3DC38
:101F90000C5F0C3019F08FEF8093600000936100AC
:101FA00084E190B3947831F48150D9F71092810094
:101FB00010927B00103118F08699105104C0123035
:101FC00010F0869B125011114CCE3BCEE199FECF02
:101FD0009FBB8EBBE09A99278DB30895262FE19978
:101FE000FECF9FBB8EBB2DBB0FB6F894E29AE19A51
:101FF0000FBE01960895F894FFCFFF5A1E93070075
:00000001FF
